:030000000210D912
:0C10D90078FFE4F6D8FD7581DB021120E1
:01003A0022A3
:061A3E008B538A54895508
:101A44007577027F48121B7C121D9CEF20E0F9ABD6
:101A540053AA54A955120830787DE6FE08E6FDED38
:011A6400FF82
:011A6500225E
:100EC500434647002D53322D0052415445434C5261
:100ED50020554E49544C495445545249475452455E
:100EE500565354525453544F505A4355545A5431EF
:100EF500205A5432205A45524F4241554444464C9B
:100F0500545341564552535420504320205F3120BD
:100F1500735F3220735F3520733120732032207365
:100F25002035207320313020733330207331206D0C
:100F35002032206D2035206D203130206D3330205A
:100F45006D312068200000000100020005000A0044
:100F55001400320064012C025804B00BB817704617
:100F6500508CA00102040810304665657459617201
:100F7500644D6574724F6666204F6E20204E6F205B
:100F850020596573204F6666204F66662054726946
:100F9500674F66662054726967537472745265634D
:010FA500202B
:1015D800740526F618E436F6C308E62225E0244A00
:1015E800F582E4340FF58322900F689375F018A400
:1015F800FFAEF0220555E555C39403220555E55580
:10160800C3940222A655E55575F004A42208F608ED
:04161800F608F622B8
:1016A300789D76AB0876CD08760008760AE408F6CE
:1016B30008760108F608766408764012161508F6CF
:1016C30078ABF608761E08F608763C0876010876AD
:1016D3005E08760108769012161578B87605021919
:0116E300EB1B
:10196100751E1D751FC01214FF789EE664CD7004AC
:1019710018E664AB60031216A378B7E6FFF46003C0
:0F198100EF700478B7760478B8E6B4FF02760505
:011990002234
:101C2900C2AF5387DF7DC07C1DE4FF121C5143877F
:031C390020D2AF07
:011C3C002285
:1014FF007560FF851E61851F6275630075640075D9
:10150F00659DE4FFAB60AA61A9628F8275830012AB
:10151F000803AB63AA64A9658F8275830012084222
:10152F000FBF1CE078B6E6FFF46003EF700478B6E7
:0A153F00760478B7E6B401027604E2
:01154900227F
:1019EB007D01E4FF121B41121C29C2AF5387DF7F1D
:1019FB009D7B1C7DC07C1D121C5B438720D2AF7F5F
:0A1A0B0002121890E4FDFF021B41D7
:10003E00E4F5537BFF7A0E79C51217A77F051218C8
:10004E0090A297829650FAA2969217A2979218E5CE
:10005E005375F004A424CEF9740E35F0FA7BFF121A
:10006E0017A77F05121890855354E4F5557BFF7A38
:10007E000E79C91217A7E553B40D00400302012CE7
:10008E00900095F82828730200BC02012C0200DDB6
:10009E000200E50200E90200F10200F90200FD0291
:1000AE00010D0201110201150201050201217F015C
:1000BE00EF1215E4789FE6FC08E6FD7401936D706F
:1000CE0003E4936C70028F550FBF0FE40201BB78EF
:1000DE00A1E6F5550201DA78A2800278AAE6F55576
:1000EE000201F478A9E6F55502022378B38002786E
:1000FE00B4E6F55502023D78B5E6F5550202C47830
:10010E00B1800678AB800278ADE6FE08E6FFF555C5
:10011E000202ED78B8E6F5551215F00202EDE55340
:10012E006554600302005DA217309601B35013A20E
:10013E0096921730960C0553E553C394104003E482
:10014E00F553A218309701B350D4A2979218309756
:10015E00CDE553B4100050C690016DF828287302F7
:10016E00019D0201C60201CC0201E602020002025A
:10017E001502022F02024902025E02027C0202975F
:10018E000202B20202D80202F30202F90202FF05D3
:10019E0055E555C3940F4003755501E5551215E409
:1001AE00E493FF740193789FCFF608EFF612160EC4
:1001BE00240EF9740F0202CD1213B602012C121581
:1001CE00FC4003E4F55578A1A655E55575F004A459
:1001DE00246EF9740F0202CD1216044003E4F55595
:1001EE0078A2A655E55575F004A4247AF9740F0289
:1001FE0002CD1216044003E4F55578AA12160C240B
:10020E007AF9740F0202CD1216044003E4F5557804
:10021E00A9A655E55575F004A42482F9740F0202BF
:10022E00CD1215FC4003E4F55578B3A655E555758A
:10023E00F004A4248AF9740F0202CD1215FC4003B7
:10024E00E4F55578B412160C248AF9740F0202CD17
:10025E0078B274321215DA94DC18E69405400576FD
:10026E000008766478B1E6FE08E6FF0202ED78AC8F
:10027E001215D8942C18E694014005760008760ADB
:10028E0078ABE6FE08E6FF805678AE1215D8942CB1
:10029E0018E694014005760008760A78ADE6FE0869
:1002AE00E6FF803B0555E555C394044003E4F55540
:1002BE0078B5A655E55575F004A42496F9740F3556
:1002CE00F0FA7BFF1217A702012C0555E555C394D2
:1002DE00064003E4F55578B8A655E5551215F0120B
:1002EE0012E502012C1216A302012C1219EB0201C7
:0702FE002C43A20802012CB1
:0A1D6E004552415300444F4E45001A
:101CDB00789FE6F52E08E6F52F22E50BAE0A78067F
:011CEB0022D6
:10116500C215C21678B7E6FFE4FCFDFEFB7A20F94E
:10117500F81208648F118E108D0F8C0EE47B40FAE7
:10118500F9F81208EF8E088F09E4F554F555C3E513
:10119500559509E5549508501CE55364816016AFD3
:1011A50055AE54121991121C3D8F530555E55570D6
:1011B500DD055480D9E553B48108E5551555700210
:1011C5001554E55565097004E5546508700CD2158C
:1011D500121D3AE4F50AF50B800785540A85550B6F
:0B11E500E4F50CF50D752D80121CDBED
:0111F00022DC
:10199100C3EF9509EE95085024EF7806C333CE3393
:1019A100CED8F9FD757702EE787DF6CFEDCFEF0851
:0D19B100F67F50121BFD121D9CEF20E0F987
:0119BE002206
:031BB200CDEFCDA7
:101BB500757702EE787DF6ED08F67F50121BFD1263
:061BC5001D9CEF20E0F979
:011BCB0022F7
:101C3D007577017F50121B7C121D9CEF20E0F97807
:031C4D007DE6FF32
:011C50002271
:101C1400121BB2E4FFFE0FBF00010EBE0FF8BFA0FF
:041C2400F5121C3D5C
:011C28002299
:0618C600CBEFCBCAEECA15
:1018CC00301503301627757703EA787DF6EB08F6AA
:1018DC0008EDF67F50121BFD121D9CEF20E0F9E481
:0D18EC00FFFE0FBF00010EBE0FF8BFA0F5FC
:0118F90022CC
:1016E40075560075570075582DE4F555121CE5C361
:1016F40033CE33CED8F97C002555FFEC3EFEAB56F5
:10170400AA57A958855582758300120803FD12183B
:10171400C60555E555C3940640D2750C00750D06F3
:0117240022A2
:10126D008E538F54121CE5C333CE33CED8F9250DD2
:10127D00FFE50C3EFEEEC0E0EFC0E0E553FDD0E033
:10128D00FFD0E0FE1218C6050DE50D7002050C121B
:10129D001CE5C333CE33CED8F9250DFFE50C3EFE4C
:1012AD00AD541218C6050DE50D7002050C0531E59E
:1012BD003170020530C3E50D9440E50C94004017E4
:1012CD00E4F50CF50D050BE50B7002050A9509E526
:0812DD000A95084002D2152217
:1013B600E4F50CF50D7BFF7A1D796E1217A7D21690
:1013C600E4F560F561C3E5619509E560950850218E
:1013D600E561AE607806C333CE33CED8F9F50D8E0F
:1013E6000C7D81FF1218C60561E56170D805608025
:1013F600D4C2167BFF7A1D79731217A7E4F50AF596
:071406000BF50CF50DC215FA
:01140D0022BC
:10135D00E4F560F561F562F563C3E5639509E56252
:10136D0095085044E5616481603EAF63AE62121929
:10137D0091121C3D8F61E56164807022AF60056044
:10138D00FCFDFEFBFAF9120BA17F2C121DA2AE6221
:10139D00AF63E4FCFDFBFAF9120BA1121D8C056382
:0813AD00E56370B5056280B133
:0113B5002215
:02154A008F60B0
:10154C00E4F561F562F563F564C3E5649509E5635B
:10155C0095085030E5626481602AAF64AE6312195D
:10156C0091121C3D8F62E562B4800FE5616560707D
:10157C0007AF64AE6302199105610564E56470C937
:04158C00056380C5AE
:011590002238
:10172500121CDB78AAE6F532E4F530F5311216E441
:10173500850A12850B137F01121AB430021A78AD8F
:10174500E6FE08E6FFE4FCFD7B64FAF9F81208649E
:101755008F4D8E4C8D4B8C4A300505C205121BE50D
:011765002261
:1017E700850A53850B54E50D450C60080554E554EF
:1017F7007002055385120A85130B1216E485530AE6
:1018070085540BC3E5549509E55395084007E4F55E
:0A1817000AF50BD2157F02021AB485
:101C5100740478FF769612FF0322740078FF76965B
:041C610012FF032249
:03003300020DD2E9
:100DD200C0E0C0F0C083C082C0D0E8C0E0E9C0E09B
:100DE200EAC0E0EBC0E0ECC0E0EDC0E0EEC0E0EF56
:020DF200C0E05F
:100DF400E5D954F8FF1209CA0E21080E21100E304D
:100E0400180E4B200E32280E4B300E4D380E534028
:100E14000E4B480E6C500E895800000E97857ADAF6
:100E2400C2DDC2DC7578007579008070800EE577CC
:100E3400700280560579E5797002057812000E8FEC
:100E4400DAC2DDC2DC80558016D2DDC2DC804DC240
:100E5400DDC2DCE5777004C2DA8041D2DA803DC2BB
:100E6400DDD2DC7575048034AFDA121D560579E5E0
:100E74007970020578C2DDC2DCE5777004C2DA80DD
:100E84001BD2DA8017AFDA121D56C2DDD2DC7575BB
:0E0E9400028009757504C2DDC2DCD2DAC2DB51
:100EA200D0E0FFD0E0FED0E0FDD0E0FCD0E0FBD00F
:100EB200E0FAD0E0F9D0E0F8D0D0D082D083D0F000
:030EC200D0E0324B
:1019BF0043910C43920CE4F5DBEF25E0F5DB301798
:1019CF000343DB0175DD1775DC1775D84453F8FE3B
:0C19DF0053F7FE43F701E4F575D2E8224F
:101BFD00E57530E002FF22E4F576757503EF25E01B
:071C0D00F57AD2DD7F02220F
:101B7C00E57530E002FF22E4F5761577757505EF13
:0B1B8C0025E04401F57AD2DD7F022243
:061D9C0020DBFDAF752203
:0D000E001577AF760576747D2FF8E6FF229A
:0C1D5600747D2576F8EFF60576157722EF
:0D0026007584C075853F53913F759200228F
:10159100C3E49515F517E49514F51622C3E51595E1
:1015A1002BF51AE514952AF51922E52B9515F51A4F
:1015B100E52A9514F51922D3E52B9515E52A9514FD
:1015C10022C3E51A94B8E519940022C3E4952BF5DA
:0715D10017E4952AF516222C
:101B0000E4F593758640F5944384405385BF53F8BC
:101B1000FD53F7FD43F80243F702F518C20CD2E972
:011B200022A2
:03003B000209F0C7
:1009F000C0E0C0F0C083C082C0D0E8C0E0E9C0E081
:100A0000EAC0E0EBC0E0ECC0E0EDC0E0EEC0E0EF3B
:100A1000C0E0308610C20C758D00758B00D28E75CB
:100A20009402020B7BC28EAF8DEFAD8BF514EDF50A
:100A3000150518E549B407004003020B6D900A4400
:100A4000F8282873020A59020A72020AB4020B0C2F
:100A5000020B21020B3B020B55121591E518C394B2
:100A6000645003020B6D85142A85152B754901020C
:100A70000B061215911215B840051215AB80031222
:100A8000159DD3E51A94E1E519940240250544E546
:100A900044940A5003020B6D754400753A00753B8F
:100AA00000754902121BE5753300753400D20E0241
:100AB0000B6D8052121591C3E53B78AC96E53A1860
:100AC00096501678B1E6FE08E6FFC3E5349FEE6463
:100AD00080F8E5336480984010C28275280075293B
:100AE00000754903D20D020B6D1215B840051215A1
:100AF000AB800312159D1215C2500B0544E544C38B
:100B0000940A40698030754400020B6D1215CCC305
:100B1000E52978AE96E52818964052754904020BEF
:100B20006D1215CC1215B840051215AB80031215C5
:100B30009D1215C250377549058032121591C3E5D3
:100B4000349432E533648094805022754906D21083
:100B5000121D6280181215911215B840051215ABBE
:100B6000800312159D1215C25003754901E516F553
:100B70008D85178BD287D28E7594005394FED0E06A
:100B8000FFD0E0FED0E0FDD0E0FCD0E0FBD0E0FA0A
:100B9000D0E0F9D0E0F8D0D0D082D083D0F0D0E04F
:010BA0003222
:0F1D0D00AF49121BCCAF15AE14121CEC021D8C8B
:101A8D006F035D5733767E437F771004007B3E6C8A
:101A9D001F7C78773B020F382C5A1A6F79751876A0
:071AAD003C0E2F4E2B375DAC
:10192E004EFECCEFCC0F747D2CF8EEF6EDC43322C8
:10193E00901A99E493FF78D1F608EFF608F608F6B8
:10194E0022E493FF74D12EF8EFF60E22EE3395E0DB
:03195E00FDFC226B
:10104600E4FF0F247DF876CD0F747D2401F87680B9
:101056000F747D2402F876E00F747D2403F876F889
:1010660030190A0F747D2404F87671800ACEEFCE0B
:101076000F747D2EF8767078D1E6FEC4540FFDCC41
:10108600EFCC0F747D2CF8EDF6EEC454F0FE78D25A
:10109600E6FD131313541F12192E54E0FE78D3E6FF
:1010A600FD1313543F12192E3354C0FE78D4E6FDB7
:1010B600C31312192E33335480FECDEFCD0F747D3A
:1010C6002DF8EEF68F777F38121BFD121D9CEF2050
:0210D600E0F93F
:0110D80022F5
:1018FA00C21912193E75770A787D76CD0876800866
:10190A0076E00876F80876700876050876D50876BF
:10191A009B0876FFE408F67F38121BFD121D9CEF28
:03192A0020E0F9C1
:01192D002297
:101B9700EF24F9600B14600C2402700EC219800741
:0B1BA700D219800312193E12104622D2
:10140E00C3EF648094E1400ED3EF648094FA5006EB
:10141E00EF24ACFF803CC3EF648094C1400ED3EF49
:10142E00648094DA5006EF24CCFF8026C3EF6480EC
:10143E0094B0400ED3EF648094B9500674D02FFF51
:10144E008010BF2D047F0A8009BF5F047F0B8002CE
:03145E007F0C22DE
:101A6600CEEDCECDEFCDCFEECF12140EEF3395E007
:101A7600FE748D2FF582741A3EF583E493FF74D1BC
:071A86002DF8EFF6021046F7
:0617A7008B628A63896475
:1017AD00E4FE901A9912194FBE04F7E4FEAB62AA3B
:1017BD0063A9648E82758300120803FF60191214E9
:1017CD000EEFFD3395E0FC748D2DF582741A3CF50A
:0A17DD008312194FBE04D602104615
:0412E5008F828E83E3
:1012E90012195A7B197AFC79FF78FFD312098F40BA
:1012F9000390FC19AF82AE8312195AE47B0F7A2747
:10130900F9F8C312098F500390270FE4F55674CCEE
:101319002556F8E4F60556E556B405F2AE83AF82D4
:1013290012195A7B007A0079CC120BA178CFE6709A
:101339001A75560374CB2556F8E6FF74CC2556F872
:10134900EFF6D556EF78CC762080E17B007A0079EC
:04135900CC0217A704
:101CB500C212C214C211E4FDFF121B41E4FD7F01F3
:031CC500021B41BE
:101B4100EF146011047016BD0104C2828002D282BA
:0E1B5100A282921322BD0103C28122D2812200
:101AB400EF24FE600D14601124027019D212751CFB
:101AC4000122C212A213928222D214751D027D0138
:061AD4007F01121B4122FC
:101A1500301212D51C0F308207C282751C0F80054B
:101A2500D282751C23E51DD39400400CD51D09C237
:091A350014E4FD7F01121B4122A3
:0F1D2B0046554C4C005A46354A0020342D3400A2
:030036000135632E
:0A1D7800E4F543F542F541F5402281
:021890008F6166
:10189200E4F562F563C3E5639561E5629400502364
:1018A200900000AF82AE83E4FCFD7B207A4EF9F813
:1018B200D312098F4003A380EA0563E56370D6055E
:0318C2006280D26F
:0118C5002200
:0E1D3A007BFF7A1D792B1217A77F0A021890E3
:0F1D1C00D20B301506121D3AC20B2212172522C8
:05001E00C20B0217E710
:0C1D6200121D78F527F526F525F5242242
:101BE500121D78853F27853E26853D25853C24F5B4
:081BF5003FF53EF53DF53C22F1
:101CFD008E7B8F7CEEFF121DA2AF7CE57C021DA2B8
:10030500120026121D82121CB57F04121890209728
:100315000B7D057F011211F1D2AF80FE209612D21E
:10032500AF121961C2177F701219BF121165120041
:100335003E12196178B8E6FDE4FF1211F1438720FA
:10034500D2AFC2177F701219BF7F01121890121118
:10035500651218FA7A1D793012059F7A1D793512C2
:10036500059F12003AE478DBF61217667F01121832
:1003750090121DA5A2969208A2979209E4F54EF552
:1003850039F538F537F536F54F7543F17542D875BA
:1003950041FF7540FFF527F526F525F524C20AF539
:1003A5003FF53EF53DF53CC20BF550F551C20DF557
:1003B5002078A2E66004D2808002C28078B5E62467
:1003C500FE600B14600C2402700AD2038006D2046E
:1003D5008002D205E4F549752C64C20EC210121BC9
:1003E5000078DBE6C3940240F8E4F6D52C19752CA9
:1003F500647402253BF53BE4353AF53A7402252948
:10040500F529E43528F528300E07C20ED20B121D4A
:100415001C301007C210C20B12001E209605209733
:1004250002D20FA208309601B3501AA29692083054
:100435009613200F10300A06C20A7F068004D20ADE
:100445007F07121B97A209309701B35004A2979218
:10045500091205AA054FE54FC39401500302058D06
:10046500E4F54FFB7A007952121A3E78D5EEF6087C
:10047500EFF6E5526402600302058D78D5E6FE08C5
:10048500E6FF78A1E6FD1214B3E5392FF539E53815
:100495003EF538E5373DF537E5363CF536054EE5AD
:1004A5004EC39405500302058DAF39AE38AD37AC58
:1004B50036E47B05FAF9F812161C8F398E388D371C
:1004C5008C36C3E5399527F539E5389526F538E5B0
:1004D500379525F537E5369524F536AF43AE42AD6C
:1004E50041AC40AB39AA38A937F8D312098F400C73
:1004F500853943853842853741853640300A0AAF0C
:100505004378D7E542F608EFF6AE38AF3978D5EE41
:10051500F6FE08EFF68E33F534300A0308800278CC
:10052500D5E6FE08E6FF1212E50551E55170020514
:1005350050C378A096E5501896402EE4F550F55135
:10054500300B267F03121AB4201518300D097F00D1
:100555007E8212126DC20D78D5E6FE08E6FF1212F4
:100565006D8006121D3A12001E85393F85383E857D
:10057500373D85363CE4F539F538F537F536F54E32
:10058500300405C204121BE5E53565496006854959
:0A05950035121D0D121A150203E6BF
:0B059F007BFF1217A77F0412189022A8
:101ADA00444C0021536967005A46354A004D4F4429
:101AEA0000342D34004170722032302032303038C8
:061AFA000050524F4700AE
:10166000AF5BAE5AAD59AC58EC4D4E4F22EF24FF54
:10167000F55BEE34FFF55AED34FFF559EC34FFF528
:101680005822E4755B20755A4EF559F55822E475D9
:101690005B01F55AF559F5582275550075560075D8
:0316A000579D2231
:1005AA00121D48EF70030207CA121B5FEF1209CA35
:1005BA0007A32407AE2A07984D07B35006F0520541
:1005CA00E56106756307C76406CB7206C87306F44D
:1005DA0074076876076378000007CAC20A7BFF7A45
:1005EA001A79DA1217A7121682121D48EF700A1228
:1005FA001660600512166D80F0121660700302070D
:10060A00CA121B5F8F5412154AE4F55B121692E464
:10061A007F06FEFDFCAB5BAA5AA959A858C312096A
:10062A00A5501F121C3D8F54121DA2E55B2401F533
:10063A005BE4355AF55AE43559F559E43558F55815
:10064A0080CD121C3D8F54E55464806016E55464D5
:10065A00816010121DA2121C3D8F54121DA27553E7
:10066A00018003E4F553E55370D822121699121645
:10067A008EF5541216606024121682121D48EF700D
:10068A000A121660600512166D80F0121660600379
:10069A001207CB0554E554C3941C40D71216606068
:1006AA001A789DB6AB0708B6CD030207AB7BFF7A73
:1006BA001A79DD1217A77F0A02189002076002133F
:1006CA005D121699E4F554AB550557E557AA5670CD
:1006DA0002055614F91207EAFF121DA20554E55441
:1006EA00C3941C40E22243A20822C20A755500752F
:1006FA0056007557D912168EF554121660602412D8
:10070A001682121D48EF700A121660600512166DE5
:10071A0080F012166060031207CB0554E554C394A7
:10072A000240D7121660602E78D9E6FE08E6FFEE80
:10073A003395E0FDFCC3EF953FF55FEE953EF55E20
:10074A00ED953DF55DEC953CF55CAF5F78A7E55E10
:10075A00F608EFF6804B0214FFC20A0213B67A1AA1
:10076A0079E21207DF7A1A79E7121CC878B6E6240A
:10077A0030FF121DA2121D8C7F76121DA27A1A79E1
:10078A00EB1207DF7A1A79EF121CC8021D8CE4F506
:10079A0054435401AF54021DA2C20AE478A7F608D2
:1007AA00F60219EBC20A0216A3C20A7BFF7A1A7969
:1007BA00FB1217A77D017F011211F180FE121D0D98
:1007CA0022121B5FAB55AA56A9578554827583001E
:1007DA00EF120842227BFF121CC8121D8C7BFF22DB
:0A1D8200E4F5955396BF53A27F22AB
:101766005389F0438901538FFE758C70E4F58A53D3
:10177600B8FD53B7FD43B702D2A9D28C53890F43A4
:101786008910538FEFF58DF58B53847F43858053F6
:10179600A2DF53B8F743B80853B7F743B708D2AB3D
:0117A6002220
:03000B00021C656F
:101C6500C0E0E8C0E078DB06758C70758A00D0E0CE
:041C7500F8D0E03291
:03001B00021D952E
:071D9500C287C28ED20C329E
:101C79000D0A003031323334353637383941424371
:041C89004445460088
:101C8D00AF74AB68AA69A96A057422AF67AE66AD79
:041C9D0065AC6422AC
:1011F1005387BF75985053877FE4F5BABF01054304
:10120100A240800353A2BFE4F5BDED146015146044
:101211001A14601F1460242404702575BEF075BF74
:101221000B802375BEF075BF05801B75BEF075BFC1
:1012310002801375BE7075BF01800B75BEB080034F
:1012410075BE30E4F5BF75BD035391FE4392014372
:1012510091025392FDC21A53B8EF53B7EF43B8103E
:0C126100E478CAF618F678CBF6D2AC227E
:0300230002185967
:10185900C0E0C0D0E8C0E030981E78CAE6C3940F53
:10186900501418E60624B9F8A69978CA0618E6C3EA
:10187900941040027600C298309904C299C21AD0D5
:07188900E0F8D0D0D0E032FE
:08000300201AFDD21A8F992288
:101B210078CAE6D39400401508E60624B9F8E6FF22
:0F1B310078CA1608E6C394104005E4F6227F0038
:011B40002282
:031DA20002000339
:101B5F007F207E4E78CAE67010D3EF9400EE94008B
:0C1B6F004007EF1F70EE1E80EB121B21E0
:011B7B002247
:101CC8001207EAFF600C121DA2740129F9E43AFA1E
:031CD80080EE2279
:0E1D480078CAE6D3940040037F01227F002278
:101BCC00CEEFCEEE54F0C4540F901C7C93FF121D3C
:091BDC00A2EE540F93FF021DA2BA
:101CEC00CDEFCDCCEECCEEFF121BCCCFEDCF021B4B
:011CFC00CC1B
:091D8C007BFF7A1C7979021CC866
:0E0BA1008F678E668D658C648B688A69896AA1
:100BAF00E4F574EC4D4E4F7017E94A4B70057F30EA
:100BBF00021DA2121C8D8F827583007430020CC42B
:100BCF00121C9AEC33502AE56A4569456870077F15
:100BDF002D121DA2800D121C8D8F82758300742D16
:100BEF00120842121C981209818F678E668D658CD0
:100BFF0064757301756E00756DCA756C9A756B3B74
:100C0F00E4FFFEFDFCAB6EAA6DA96CA86BD31209B5
:100C1F00A55003020CAF121C98A86B1208EF8F722D
:100C2F008E718D708C6FEC4D4E4F7004E573702389
:100C3F00E5722430FFE56A456945687005121DA20B
:100C4F00800EAE74121C8F8E82758300EF120842D5
:100C5F00E4F573AF6EAE6DAD6CAC6BAB72AA71A9F0
:100C6F0070A86F120864CAEECAC9EDC9C8ECC8C330
:100C7F00E5679FF567E5669AF566E56599F565E5BC
:100C8F006498F564AF6EAE6DAD6CAC6BE47B0AFA35
:100C9F00F9F81208EF8F6E8E6D8D6C8C6B020C0F46
:100CAF00E569456A45686010AB68AA69A96A8574E9
:080CBF0082758300E412084273
:010CC700220A
:100FA600308F426831D1407433173E8034633C8CB5
:100FB60035B13A98370938A4386636B039C734BCE3
:100FC6003B2D32C83C9D30D43E0F2EE03F882CECA2
:100FD60041062AF8428D29044418271045AB251CE2
:100FE6004741232848E121344A861F404C311D4C95
:100FF6004DE21B584F9C1964515D17705323157CA5
:1010060054EF138856C4119458A20FA05A830DACFE
:101016005C6D0BB85E6009C4605807D0625A05DC87
:10102600646203E8667301F4688A00006AA1FE0C34
:101036006CB8FC186ECFFA2470E6F8300000000099
:10182100F583E493FE740193FFE55A25E025E02258
:10183100F583C37401939FFFE4939EFEE4228F5BC3
:101841008E5A8D598C58228F578E568D558C542215
:0818510024A6F582E4340F2205
:101CA100C3EF9DEE9C400AD3EF9BEE9A50037F0158
:041CB100227F00226C
:040CC8008E588F595A
:100CCC00E4F55A12182A121851F583E493FC7401B6
:100CDC0093FD12182A24AAF582E4340FF583E493C9
:100CEC00FA740193FBAF59AE58121CA1EF700302BA
:100CFC000DC012182A12185112182124AAF582E4D8
:100D0C00340F1218318F5E8E5DF55CF55B12182A6C
:100D1C0024ACF582E4340F12182124A8F582E434B3
:100D2C000F1218318F628E61F560F55FAD60AC5FAC
:100D3C001209818F628E618D608C5FAE58AF59E461
:100D4C00FCFDEEC0E0EFC0E012182A121851F5833A
:100D5C00E493FE740193FBCAEECAD0E0FFD0E0FE30
:100D6C00C3EF9BFFEE9AFEED9400FDEC9400FCAB00
:100D7C0062AA61A960A85F120864AB5EAA5DA95C57
:100D8C00A85B12161CC8ECC8C9EDC9CAEECACBEFD9
:100D9C00CB12182A24A8F582E4340FF583E493FED1
:100DAC00740193FFE4FCFDEB2FFFEA3EFEED39FDF1
:100DBC00EC38FC22055AE55AC394275003020CCF99
:050DCC00E4FFFEFDFC48
:010DD10022FF
:011DA500221B
:1014610012183FAB5BAA5AA959A858E8C0E078A561
:10147100E6FE08E6FFE4FCFDD0E0F812086412186D
:101481003F780E1209B612183F78A7E6FE08E6FF6C
:10149100EE3395E0FDFCE55B2FF55BE55A3EF55A31
:1014A100E5593DF559E5583CF558AF5BAE5AAD5994
:0214B100FC221B
:0214B3008D5357
:1014B500120CC8121848121461121848E55314602A
:1014C5001C14702DE47FE87E03FDFCAB57AA56A9DA
:1014D50055A854120864E47BE87A0B800CAF57AE2C
:1014E50056AD55AC54E47B03FAF9F812161C1218E4
:0914F50048AF57AE56AD55AC549A
:0114FE0022CB
:1010E500020305E493A3F8E493A34003F68001F219
:1010F50008DFF48029E493A3F85407240CC8C3330C
:10110500C4540F4420C8834004F456800146F6DFDA
:10111500E4800B0102040810204080900036E47E34
:10112500019360BCA3FF543F30E509541FFEE493CF
:10113500A360010ECF54C025E060A840B8E493A396
:10114500FAE493A3F8E493A3C8C582C8CAC583CAC1
:10115500F0A3C8C582C8CAC583CADFE9DEE780BE79
:0100390000C6
:1007EA00BB010689828A83E0225002E722BBFE020D
:0907FA00E32289828A83E4932240
:10080300BB010CE58229F582E5833AF583E02250AA
:1008130006E92582F8E622BBFE06E92582F8E222F4
:0D082300E58229F582E5833AF583E493220E
:10083000BB010689828A83F0225002F722BBFE01A7
:02084000F322A1
:10084200F8BB010DE58229F582E5833AF583E8F0EC
:10085200225006E92582C8F622BBFE05E92582C898
:02086200F22280
:10086400E88FF0A4CC8BF0A42CFCE98EF0A42CFC33
:100874008AF0EDA42CFCEA8EF0A4CDA8F08BF0A4B1
:100884002DCC3825F0FDE98FF0A42CCD35F0FCEB10
:100894008EF0A4FEA9F0EB8FF0A4CFC5F02ECD39D5
:0F08A400FEE43CFCEAA42DCE35F0FDE43CFC2242
:1008B30075F008758200EF2FFFEE33FECD33CDCCFC
:1008C30033CCC58233C5829BED9AEC99E58298407F
:1008D3000CF582EE9BFEED9AFDEC99FC0FD5F0D65C
:1008E300E4CEFBE4CDFAE4CCF9A88222B800C1B986
:1008F3000059BA002DEC8BF084CFCECDFCE5F0CBC4
:10090300F97818EF2FFFEE33FEED33FDEC33FCEBFC
:1009130033FB10D703994004EB99FB0FD8E5E4F9B7
:10092300FA227818EF2FFFEE33FEED33FDEC33FCA4
:10093300C933C910D7059BE99A4007EC9BFCE99A98
:10094300F90FD8E0E4C9FAE4CCFB2275F010EF2FDD
:10095300FFEE33FEED33FDCC33CCC833C810D707DD
:100963009BEC9AE899400AED9BFDEC9AFCE899F818
:0E0973000FD5F0DAE4CDFBE4CCFAE4C8F922AB
:10161C00C2D5E830E70FB2D5E4C39BFBE49AFAE4F9
:10162C0099F9E498F8EC30E717B2D5121652120873
:10163C00EFE4C39BFBE49AFAE499F9E498F880038D
:10164C001208EF30D50DE4C39FFFE49EFEE49DFD30
:04165C00E49CFC22EC
:0E098100C3E49FFFE49EFEE49DFDE49CFC2287
:10098F00EB9FF5F0EA9E42F0E99D42F0EC6480C8DF
:06099F0064809845F0227F
:1009A500EB9FF5F0EA9E42F0E99D42F0E89C45F0A8
:0109B500221F
:1009B600E86010ECA2E713FCED13FDEE13FEEF1357
:0409C600FFD8F02244
:1009CA00D083D082F8E4937012740193700DA3A3BC
:1009DA0093F8740193F5828883E4737402936860D0
:0609EA00EFA3A3A380DFD0
:00000001FF
